:080000002DC0FECFFDCFFCCFA7
:10000800FBCFFACFF9CFF8CFF7CFF6CFF5CFF4CFB4
:10001800F3CFF2CFF1CFF0CFEFCFEECFEDCF102768
:10002800E80364000A00010000100001100001004C
:1000380020456E61626C6564204F555425752E0D00
:10004800002044697361626C6564204F55542575BE
:100058002E0D0000F894EE27ECBBE5BFF8E1A4B73D
:10006800A77FA4BFF1BDE1BD8DE0A2E0ED938A9525
:10007800E9F780E8A0E6ED938A95E9F7E0E0E3BBCD
:10008800E0E0E4BBE0E0E5BBEFEDEDBFC0E8D0E0C9
:1000980000C0E0E8E6BDE0E0E6BDEBBBEABBE8BBDC
:1000A800EFE0E7BBE0E0E2BBE1BBE0BFE3BFE2BFFC
:1000B800E6BFECBFEFBDEEBDEDBDECBDE5BDE4BDFB
:1000C800EBBDEABDE9BDE8BDEBBFE5BFE9BFEDB9F2
:1000D800EBB9E8E1EAB9E6E0E3B9E0E0E2B9EFE27A
:1000E800E9B9E0E8E8B9C498E0E0E8BB3324E4E023
:1000F8003E16A0F4E4E6F0E0C8D117D2E32DA8E05C
:1001080024D2E8BBE8E3F0E0C3D1ECEDF5E0BDD1E3
:100118000CD2E9E4F0E0BCD13394E9CFE7CFFFCFCC
:100128005D9BFECFE881ECB9219608951A93AA81C8
:10013800EC91E03089F0A981EC911E2FE03021F09C
:10014800123048F011501C93AA81EC91EF5FEC93A8
:10015800E150AB81A08303C0EB81EA93E1DF188112
:100168002496089526972ED210E0EF85F8893196C7
:10017800EF87F88B3197E4912E2FE03009F454C1C2
:10018800E12F90D1309731F4253211F411E001C0FC
:100198008BD149C1E130A0E0FA07A1F4253211F46E
:1001A80083D140C112E040E000E02D3211F401E0BB
:1001B8003AC12B3211F44BE236C1203211F440E23D
:1001C80032C104C0E230A0E0FA0751F450E013E075
:1001D800203329F470D1E0E8F0E070D124C105C0E3
:1001E800E330A0E0FA0709F01EC1203310F02A33EB
:1001F80008F013C0A52F65D1EAE0F0E0BED15E2F6C
:10020800652F7727A22F5DD1E0E3F0E0D4D1EA1B78
:10021800FB0BDB01EA0F5E2F06C1E22F43D1E33669
:10022800A0E0FA0731F44FD1EE85A481AA934FD10B
:10023800F9C0E337A0E0FA0741F445D14ED1EC917B
:10024800EE83EA930ED11E2F10C0E037A0E0FA0724
:10025800B1F439D142D1A2D143D145D116D10AD175
:100268001E2F29D1E8E0F0E029D125D1E2E0F0E025
:1002780025D121D1EFE7FFEF39D130E041C0E43695
:10028800A0E0FA0721F0E936A0E0FA0721F413D13B
:1002980030D114D104C0E537A0E0FA0729F4E6E22A
:1002A800F0E01ED115E012C0E835A0E0FA0729F405
:1002B80002D1E8E0F0E002D105C0E837A0E0FA0793
:1002C80009F0B0C0E0E3F0E00BD114E0F4D014D1B1
:1002D80099F0F9D002D162D114D1AB85AA232AF4BE
:1002E800EA85FB852ED10DD14DE2403011F01F5F1C
:1002F80002C0E1D009D104C0E6D0EFD04FD101D17E
:1003080006D199F4151788F4D6D005D151F0D3D079
:10031800F3D029F0D0D0F8D0242F115001C020E319
:1003280001C020E2C1D05150EDCF312FC4D0E2E05E
:10033800F0E0F7D0C1F03030A9F0BDD0E8E0F0E04F
:10034800F0D031F0D0D03196CBD03197E49103C0C2
:10035800AE81ED91AE83EA93BAD0503009F0515096
:100368003150E9CF56C020E3BED01CD1E887F987C9
:10037800BAD03296B5D0E885F985AA85BB85AE177F
:10038800BF0748F02F5FA885B985EA85FB85EA1B7A
:10039800FB0BB7D0F0CF2A3368F08DD0E8E0F0E05F
:1003A800C0D021F0E22F7ED0379603C0E22F7AD05A
:1003B800B7962E2F80D0E0E1F0E0B3D001F52133DD
:1003C80020F4A885B985119709F40AC0531710F0CD
:1003D8009ED009F018C020E26ED09DD081F020E3B5
:1003E800A02F6FD0E0E1F0E069D065D085D039F07A
:1003F80062D08AD04A936BD0503009F0515054D013
:10040800503009F051503150A885B985129708F03D
:10041800AACF7DD039F0503029F05150E0E2EA936C
:1004280056D0F9CF10E0A1CED4D061960895FF92AE
:10043800F82E21971A93AC2FA250AF0D1A2FE0E097
:10044800E983AC2FAE5FAF0DA9D01FD01A93EC2F64
:10045800EC5FEA93E0E0EA9385DE18812296FF904C
:100468000895BB27A991EE276D91662311F0E395B6
:10047800FBCF0895AA27BB27E991F99105900020A1
:1004880011F01196FBCFFD010895FA93EA930895B0
:10049800FCDFE32DF0E0319660D088D084E0C7DF40
:1004A80026960895F0E008952A93EE85EA93EC2FB6
:1004B800E25FEA933BCEA02FB0E00895EA2B0E2F1F
:1004C8000895B0E00895EE85E450EE870895EE852E
:1004D800EA93EC2FE25FEA9329CEAE85AC5F0895EC
:1004E800EE83FF830895EE81FF810895EA230E2F9E
:1004F8000895E4E0F0E00895FCDFEA23FB23309759
:100508000895EA87FB870895EBEFFFEFEFCFE02F21
:10051800C9DFE1700895E0E8F0E0EA23FB233097B3
:100528000895EA23FB2330970895E991F9913096CD
:1005380039F083E397E00197F1F7A8953197C9F768
:100548000895F195E195F0400895EE230E2EEA2FD7
:1005580019F0E6950A94E9F708956F2F660F660B70
:10056800762F08950A2EAA1BB9E003C008F4A00D3F
:10057800A695E795BA95D1F7089504D0F3DF0EF460
:10058800E1950895E894E7FF02C0E1956894A7FF14
:1005980004C0A19500F8039400FA0895ED91FC9128
:1005A800AA9508950590F491E02D08957A936A9399
:1005B800FA93EA9308951B2EBF2FF12D1A2EAE2F12
:1005C800E12D08955A934A933A932A931A930A93DA
:1005D80008955D814C813B812A81198108810895A4
:00000001FF
